:020000040800F2
:1000000060230020110100083502000831020008B9
:100010003302000885010008030500080000000005
:100020000000000000000000000000008503000840
:1000300087010008000000005F0200088703000835
:100040002B0100082B0100082B0100082B010008E0
:100050002B0100082B0100082B0100082B010008D0
:100060002B0100082B0100082B0100082B010008C0
:100070002B0100082B0100082B0100082B010008B0
:100080002B0100082B0100082B0100082B010008A0
:100090002B0100082B0100082B0100082B01000890
:1000A0002B0100082B0100082B0100082B01000880
:1000B0002B0100082B0100082B0100082B01000870
:1000C0002B0100082B0100082B0100082B01000860
:1000D0002B0100082B0100082B0100082B01000850
:1000E0002B0100082B0100082B0100082B01000840
:1000F0002B0100082B0100082B010008DFF80CD0B1
:1001000000F02EF800480047110D00086023002081
:100110000648804706480047FEE7FEE7FEE7FEE7A1
:10012000FEE7FEE7FEE7FEE7FEE7FEE78D030008D9
:10013000FD00000830B50B460146002020220124B6
:1001400009E021FA02F59D4205D303FA02F5491BA5
:1001500004FA02F52844151EA2F10102F1DC30BDBB
:10016000064C074D06E0E06840F0010394E8070004
:1001700098471034AC42F6D3FFF7C4FF804A00081A
:10018000A04A0008FEE77047F0B5CB7803F00F02F5
:100190001B0644BF8B781A430B881C061CD00368CF
:1001A000012400254FF00F0C202D13D00F883C4266
:1001B0000DD00CFA05F602FA05F7B3433B43CF78AE
:1001C000482F03D0282F08BF446100E004610435A4
:1001D0006400E9E703600B88B3F5807F1CD34368B4
:1001E0004FF4807400254FF00F0C202D13D00F8892
:1001F0003C420DD00CFA05F602FA05F7B3433B4337
:10020000CF78482F03D0282F08BF446100E0046155
:1002100004356400E9E74360F0BD8068084018BF1A
:10022000012070471023002A08BF1423C1507047D3
:10023000FEE7FEE7704700200021002500F0F2BC39
:100240000A681043086070472946049030463847D2
:100250002046802100F08FB8CDF8008048477047D5
:100260000149FFF7EDBF00BF1C1002400149FFF735
:10027000E7BF00BF1810024080B500F02DF8044918
:1002800004A20968C1F30311515CC84080BD00BFDE
:1002900004100240000000000000000001020304FE
:1002A0000607080970B5184E0C460546FFF7E4FF2F
:1002B0003DB13168074AC1F30221515C20FA01F1D6
:1002C000296034B13168034AC1F3C221515CC8408E
:1002D000206070BDE82A00080B49086800F003029E
:1002E0000A48022A08D10A680B68C2F38342023224
:1002F000DB0302D406485043704709685043C1F3FA
:100300004041C840704700BF0410024000127A000C
:1003100000093D0070B5026802F4415202604A894A
:100320000B884C790E7B0D7A1A434B881A430B7954
:1003300022431A43CB881A43036832432A4392B2BA
:100340001A430260C989016170BD026822F400622B
:10035000026002681143016070470021017341810E
:100360000160416001720721C1817047016841F05D
:100370004001016070478068084018BF0120704745
:10038000C1607047704700F039B9000081B0314852
:10039000314A016841F001010160416811402F4A72
:1003A0004160016811400160016821F48021016011
:1003B000416821F4FE0141604FF41F018160016832
:1003C00041F480310160002100910099090B04295A
:1003D00005D80168890302D400990131F4E7016866
:1003E000890330D51E4903230A6842F010020A60CF
:1003F0000A6863F302020A600422416821F0F001F6
:100400004160416821F460514160416862F30A2112
:100410000A224160416841F480314160416862F3E1
:1004200095414160016841F0807101600168890176
:10043000FCD54168022262F301014160416801F08C
:100440000C010829FAD107484FF00061016001B0A2
:10045000704700BF001002400000FFF8FFFFF6FEEB
:100460000020024008ED00E0BCB50446C0680D461F
:100470004EF6F3110840A97A084329890843A98850
:1004800008434CF6FF71E06020690840E9880843A2
:100490004FF6FF41206160690840A9890843606107
:1004A0005148844219BF01A8002101A90020FFF78B
:1004B000F9FE019919206FF0630348432968890008
:1004C000B0FBF1F06421B0FBF1F202FB0300322338
:1004D00003EB0010B0FBF1F000F00F0040EA021057
:1004E000A060BCBDC16841F40051C16070470068A4
:1004F000084018BF01207047426861F3080242605B
:100500007047FEE7B0B5C14D044628460221FFF70B
:1005100032FF0028F9D028462146BDE8B040FFF759
:100520002FBF00BF10B5B94CFFF792FE0028FBD1DA
:1005300010BD00BFE0B50420FFF798FE034801900E
:10054000BD4801A9FFF720FE8CBD00BF01000328B4
:1005500080B5B9480121FFF760FE002818BF0120CF
:1005600080BD00BFE0B50820FFF780FE0348019082
:10057000324801A9FFF708FE8CBD00BF04000380CC
:100580002E4804210022FFF74DBE00BF024801683B
:1005900081F00401016070470C0C014010B586B079
:1005A00044F20400FFF762FE0E480F4C0590A4F5DC
:1005B000405005A9FFF7E8FD4FF4E131002001911B
:1005C0000821ADF81000ADF80C00029020468DF81F
:1005D0000E1001A9FFF748FF2046FFF783FF06B082
:1005E00010BD00BF000203880038014006490A68B8
:1005F00010440A688242FCD3704700BF0248016879
:1006000001310160704700BF1C0000200B484FF40F
:1006100080510022FFF706BE08484FF480510122A6
:10062000FFF700BE05484FF480410022FFF7FABDF6
:1006300002484FF480410122FFF7F4BD000C014055
:10064000F8B50C46054600200021002600F0EAFA25
:10065000242000F033FBFFF7D9FF102E0AD000272B
:10066000FA2F04D0E85DFFF74DFF0137F8E7FA35C0
:100670000136F2E7FFF756FFFFF7CEFFFFF7DBFD8E
:10068000262000F01BFBFFF7C1FF102D0CD0002629
:10069000FA2E06D0A05D80F0FF00FFF733FF013691
:1006A000F6E7FA340135F0E7FFF73CFFFFF7B4FF58
:1006B000BDE8F84000F0D4BA10B50446102000F0B0
:1006C000FDFA2046BDE8104000F0E6BAB0B500F0F3
:1006D00099FA3220FFF78AFF00F09CFA3220FFF7E8
:1006E00085FF00F0CBFA28B9122000F0E7FA00F0FD
:1006F000C5FA08B10120B0BD1D4D0120A8471D4C11
:100700002720A0470120A0470120A0471120A8478B
:100710000120A0474420A8470020A0470F20A04761
:100720004520A8472720A0470120A0470020A04738
:100730000020A0473C20A8470520A0472120A8472B
:100740000020A0478020A0471820A8478020A0476D
:100750004E20A8470020A0474F20A8472720A047A9
:100760000120A04700F08AFA002818BF0120B0BD80
:10077000BD0C0008990C0008F0B585B00C20FFF7FF
:1007800075FD2148214C224F049004F5504604ADDC
:1007900030462946B8474FF400402946ADF81000CE
:1007A00048208DF813003046B8471A4804F55446DF
:1007B000FFF74AFD1848FFF747FD1848FFF744FDCB
:1007C0004FF48040FFF74CFD6D462846FFF7C5FD0E
:1007D000102029468DF80C004FF4827000904FF4E1
:1007E0004040ADF80A0000208DF808000C48019048
:1007F0002046FFF78FFD20460021FFF7A6FD20468B
:10080000FFF7B4FD05B0F0BD0001038000380040E3
:10081000890100080040038000A0038800100380C5
:100820000102000280B5FA484FF40041FFF7F5FCE1
:10083000002818BF012080BD00080140B0B5754AEE
:100840000021538A994228BFB0BD0023148AA342D5
:1008500005D2156801FB0454E0540133F6E7013179
:10086000EFE700BF2DE9F04F85B00E4607464FF089
:10087000FF304FF0FF31DDF838A0B34288BF0120D0
:1008800000900492BA421046184688BF0121029196
:100890000193981B039044BF414203910499B1EB2B
:1008A000070B48BFCBF1000B0399ABEB010980EAC2
:1008B000E071C1EBE078BCB2B5B2524620462946A1
:1008C00000F019F8B8EB490F07DC049884420FD008
:1008D000029807440398A9EB00094FEA49005845DC
:1008E000E9DC0198854203D00098D9440644E2E748
:1008F00005B0BDE8F08F0138013980B289B200F04F
:1009000055B800002DE9F8430546DDE908801C468E
:1009100016460F4658B1B9B2A14222D228463246F5
:100920000B46CDF80080FFF79DFF0137F3E7DFF8B6
:1009300038902846394632463B46FFF78DFC28461C
:1009400039462A462346FFF787FC30462146324681
:100950003B46FFF781FC304621462A462346FFF7F7
:100960007BFCBDE8F88300BF65080008B0B5294CE2
:10097000049D20600120A581628262812181E38142
:100980004D074FEAD10518BF00EBD10525820BB109
:10099000B42B02D110460A4600E00846E280A0804F
:1009A000B0BD00BF1B490860704700BF70B5194B50
:1009B000DC89B4F5877F09D05A2C0AD0B42C0FD02B
:1009C0003CBB1C89C943214404460CE00C4601464B
:1009D00009E05C89C943C0430C441989014402E021
:1009E0005C89C04304441E8AA4B201F0070089B2A6
:1009F0001B686FF0800505417443802604EBD1012C
:100A000026FA00F05C5C2043002A08BF04EA0500D7
:100A1000585470BD080000202DE9F04F89B0013016
:100A2000039080B20690C01AFA2802DD09B0BDE832
:100A3000F08F481C129D1C46082B089001D10620FF
:100A400009E0012061074FEAD40118BF00EBD4018F
:100A50006008484380B207906008DDF80C90B5FA52
:100A600085F64FF000080490A2F1200081B22C48D6
:100A700001EB4102029100EB4200019205902648F1
:100A800000EB0110009007991FFA88F08142CDD940
:100A9000082C01D1059910E0182C06D0102C0BD091
:100AA0000C2CC3D101991D4A03E00299194A01EBAC
:100AB000C10102EB810100E000990844089F4FF05A
:100AC000000B90F800A0BBF1070F0FD85FEACA70C7
:100AD0002A46B9B21FFA89F008BF7209FFF70BFF67
:100AE0000BF1010B01374FEA5A0AECE709F1010952
:100AF000082C0BD006991FFA89F0401A04998842F5
:100B000004D10898DDF80C900830089008F101082D
:100B1000B9E700BF8C1D00089C17000828130008C7
:100B2000001100082DE9F04F87B0012501F1010AFD
:100B300091464FF000085C074FEAD30418BF05EB5D
:100B4000D304461C119D53460094B0B20496039002
:100B5000B5FA85F700200099029080B2884236D21B
:100B60000021CDF8048088B248452AD2CDE905138A
:100B700010991FFA88F04FF0000B0C5CBBF1070FC7
:100B80000ED8E0072A461FFA8AF1B0B218BF7A09D8
:100B9000FFF7B1FE0BF1010B0AF1010A6408EDE762
:100BA0000136039908F10108B0B2401A4845069B86
:100BB00008BF0833049808BF064605999A460131D4
:100BC000D1E7DDF804800298C8440130C3E707B0DC
:100BD000BDE8F08F2DE9F843DDF8209098461546E2
:100BE0000E4607465C082A784AB1B8B231464346F9
:100BF000CDF80090FFF710FF27440135F3E7BDE87B
:100C0000F883000006484FF480710022FFF70ABB0A
:100C10000008014002484FF480710122FFF702BB37
:100C20000008014070B505464E200C4600F046F81D
:100C30000A4EC5F3C700B0474F2000F03FF840F21E
:100C40002710051BF92C88BF2E25E8B2B047C5F345
:100C500000203146BDE87040084700BF990C0008ED
:100C600080B5222000F02AF8F72000F015F82020A7
:100C700000F024F8BDE88040AFF3008010B544F6E2
:100C80002064FFF7CFFD28B1012024B1FFF7AEFCAF
:100C9000013CF6E7002010BDB0B50546FFF7B6FCF5
:100CA000114C29462046FFF76BFBFFF7D1FA0028CD
:100CB000FBD1BDE8B040FFF7AFBC00BFB0B5054603
:100CC000FFF7B0FCFFF7A2FC074C29462046FFF7D0
:100CD00057FBFFF7BDFA0028FBD1FFF79DFCBDE8ED
:100CE000B040FFF7A5BC00BF00380040B0B5074DCD
:100CF0000446C1B22846FFF7FFFB28468021FFF7D4
:100D0000F6FB0028F9D02046B0BD00BF00380140F6
:100D100088B000F0FBF8FFF725FCFFF70BFCFFF7AE
:100D20003DFC4948494CA0474948A0474948A0478D
:100D300049A0A0474D4801684DA000F005F950A01A
:100D4000A047FFF719FDFFF7C1FCDFF84881FF2539
:100D50007A21FA22B42300954046FFF707FEDFF818
:100D600038917A21FA22B42300954846FFF7FEFD18
:100D70004A4F4046B8474A4CFF20A0474948002602
:100D80000021FA227A23019600900020FFF7CAFE84
:100D90004846B847FF20A04743480021FA227A235B
:100DA000019500900020FFF7BDFE40464946FFF741
:100DB00047FC4FF4FA50FFF719FC4046B847FF20B4
:100DC000A0473F4D39A20A20002118230096A847CA
:100DD0003CA20A201D2110230096A84740A20A2009
:100DE000322110230096A8474846B847FF20A04765
:100DF000424800961823039040A0D0E90112C06831
:100E0000CDE90412069003AA0A204721A847012031
:100E10006721F0227423CDE900600A20FFF772FDFC
:100E200040464946FFF70CFC0120FFF745FCFFF761
:100E30008FFB10B1FFF7A4FBF9E76420FFF7D6FBA7
:100E4000FFF7A4FBF3E700BF304A0008DD100008FD
:100E50004B4A0008634A0008777777772E776561F9
:100E600063742D74632E636E0D0A0D000400002060
:100E700053797374656D436C6B3A25640D0A0000F9
:100E8000457061706572204D6F64756C65205465A6
:100E900073740D0020000020C00F0020A509000879
:100EA0003D080008F02A0008903A0008322E31333D
:100EB00020457061706572204D6F64756C6500002F
:100EC000D50B000844657369676E6564204279201C
:100ED00057654163742053747564696F00000000A6
:100EE00077697468203235302078203132322072B0
:100EF00065736F6C7574696F6E0000003E3E20482C
:100F0000656C6C6F20576F726C642E000B484FF449
:100F10007A710068B0FBF1F00138B0F1807F00D346
:100F2000FEE70749F02248600648027000228A6006
:100F300007220A6050210170704700BF04000020A2
:100F400010E000E023ED00E00FB4054B10B503A95D
:100F5000044A029800F018F810BC5DF814FB000079
:100F6000ED0C00080000002002E008C8121F08C1B4
:100F7000002AFAD170477047002001E001C1121F1A
:100F8000002AFBD1704700002DE9FF4F89B09B4636
:100F90000446002506E025280BD05A460B999047B9
:100FA000641C6D1C20780028F5D10DB02846BDE8E2
:100FB000F08F0027B8460122474900E0074314F8A4
:100FC000013F203B02FA03F00842F7D120782E2897
:100FD00019D114F8010F47F004072A280ED06FF03A
:100FE0002F022078A0F1300109290CD808EB8801E4
:100FF00002EB410100EB0108641CF2E70A98641C53
:1010000050F8048B0A9020780028CED0642808D0AD
:10101000692806D075281ED05A460B9990476D1C3A
:1010200058E00A994FF00A0901C90A91002802DA2A
:1010300040422D2102E0390504D52B218DF82010E6
:10104000012103E0F90704D02021F7E78A4608AE22
:101050000DE00021FAE70A994FF00A0901C90A9147
:10106000F7E74946FFF766F8303106F8011D00281A
:10107000F7D1ADEB060000F12009780701D44FF05D
:101080000108C84502DDA8EB090000E00020804609
:10109000002706E008A85A46C05D0B9990476D1CD2
:1010A0007F1C5745F6DB04E030205A460B999047E9
:1010B0006D1CB8F10001A8F10108F5DC05E016F897
:1010C000010B5A460B9990476D1CB9F10001A9F12B
:1010D0000109F4DC641C65E70928010010B5044629
:1010E00001E0FFF703FE14F8010B04490028F8D1D2
:1010F000BDE810400A20FFF7F9BD00000000002005
:101100000000000000000000002F000000000700A9
:10111000070000147F147F1400242A7F2A12006223
:1011200064081323003649552250000005030000CF
:1011300000001C224100000041221C000014083E57
:1011400008140008083E0808000000A0600000081D
:101150000808080800006060000000201008040271
:10116000003E5149453E0000427F4000004261512F
:101170004946002141454B31001814127F100027C9
:1011800045454539003C4A4949300001710905038C
:1011900000364949493600064949291E00003636BD
:1011A0000000000056360000000814224100001420
:1011B00014141414000041221408000201510906FD
:1011C00000324959513E007C1211127C007F49497E
:1011D0004936003E41414122007F4141221C007FAF
:1011E00049494941007F09090901003E4149497ABD
:1011F000007F0808087F0000417F41000020404137
:101200003F01007F08142241007F40404040007FA2
:10121000020C027F007F0408107F003E4141413EE6
:10122000007F09090906003E4151215E007F09192E
:1012300029460046494949310001017F0101003F2B
:101240004040403F001F2040201F003F4038403FAB
:10125000006314081463000708700807006151490F
:10126000454300007F41410000552A552A550000A2
:1012700041417F0000040201020400404040404020
:10128000000001020400002054545478007F4844B8
:10129000443800384444442000384444487F0038EF
:1012A0005454541800087E0901020018A4A4A47C18
:1012B000007F080404780000447D400000408084E2
:1012C0007D00007F102844000000417F4000007C2A
:1012D00004180478007C0804047800384444443836
:1012E00000FC242424180018242418FC007C080482
:1012F000040800485454542000043F444020003C5B
:101300004040207C001C2040201C003C4030403CE1
:10131000004428102844001CA0A0A07C0044645471
:101320004C441414141414140000000000000000B5
:10133000000000000000FC000000000002000000AF
:10134000000C020C020000000000000090D0BCD095
:10135000BC900003000300001824FE448C0003022C
:10136000070201001824D8B04C80000300010201DC
:10137000C038E438E0000102020102020806000061
:101380000000000000000000000000F8040200005F
:1013900000010204000204F8000000040201000041
:1013A0009060F86090000000010000002020FC2008
:1013B00020000000010000000000000000000806FE
:1013C000000000002020202020000000000000007D
:1013D0000000000000000002000000000080601C0F
:1013E0000200040300000000F8040404F8000102F5
:1013F000020201000008FC000000000203020000DD
:101400001884442418000302020202000804242461
:10141000D80001020202010040B088FC80000000F8
:10142000000302003C242424C40001020202010043
:10143000F824242CC0000102020201000C04E41C68
:101440000400000003000000D8242424D800010276
:101450000202010038444444F80000030202010083
:10146000000010000000000002000000000020004A
:101470000000000006000000002050880402000068
:101480000000010290909090900000000000000089
:101490000002048850200002010000001804C42447
:1014A0001800000002000000F804E494F8000102B3
:1014B0000202020000E09CF0800002030000030230
:1014C00004FC2424D800020302020100F8040404EE
:1014D0000C0001020202010004FC0404F8000203F3
:1014E0000202010004FC24740C0002030202030047
:1014F00004FC24740C00020302000000F008044401
:10150000CC4000010202010004FC2020FC04020384
:10151000000003020404FC040400020203020200AF
:10152000000404FC040406040403000004FC24D0AA
:101530000C0402030200030204FC04000000020386
:1015400002020203FC3CC03CFC0003000300030059
:1015500004FC30C4FC04020302000300F804040489
:10156000F80001020202010004FC24241800020316
:1015700002000000F8848404F8000102020705005C
:1015800004FC24649800020302000302182424448B
:101590008C000302020201000C04FC040C00000297
:1015A0000302000004FC0000FC0400010202010030
:1015B000047C80E01C040000030000001CE03CE010
:1015C0001C00000300030000049C609C0400020354
:1015D00000030200041CE01C0400000203020000DF
:1015E0000C84641C04000203020203000000FE02DB
:1015F0000200000007040400000E30C000000000DC
:1016000000010200000202FE0000000404070000C6
:1016100000040204000000000000000000000000C0
:101620000000080808080808000002000000000088
:10163000000000000040A0A0C00000010202030260
:1016400004FC2020C00000030202010000C0202092
:10165000600000010202020000C02024FC00000122
:101660000202030200C0A0A0C000000102020200AA
:101670000020F82424040002030202000040A0A07D
:10168000602000070A0A0A0404FC2020C0000203AC
:10169000020003020020E400000000020302000038
:1016A000000020E4000008080807000004FC80E0B7
:1016B00020200203020003020404FC0000000202D6
:1016C00003020200E020E020C0000300030003004A
:1016D00020E02020C00002030200030200C02020FE
:1016E000C00000010202010020E02020C000080F1D
:1016F0000A02010000C02020E0000001020A0F08D9
:1017000020E0402020000203020000000060A0A0B2
:1017100020000002020203000020F8200000000068
:101720000102020020E00020E000000102020302AA
:1017300020E0208060200000030100006080E08045
:1017400060000003000300002060806020000203AE
:101750000003020020E0208060200808070100004C
:101760000020A0602000000203020200000020DE32
:101770000200000000070400000000FF000000005D
:10178000000F00000002DE2000000004070000003F
:10179000020102040402000000000000000000003A
:1017A000000000000000000000000000000000F841
:1017B00000000000000000333000000000100C06A4
:1017C000100C0600000000000000000040C078403F
:1017D000C0784000043F04043F040400007088FC0B
:1017E00008300000001820FF211E0000F008F00063
:1017F000E018000000211C031E211E0000F00888D4
:10180000700000001E2123241927211010160E003D
:10181000000000000000000000000000000000E0E8
:1018200018040200000000071820400000020418FD
:10183000E00000000040201807000000404080F059
:10184000804040000202010F01020200000000F08F
:10185000000000000101011F010101000000000063
:101860000000000080B070000000000000000000D8
:101870000000000000010101010101010000000061
:1018800000000000003030000000000000000000F8
:1018900080601804006018060100000000E01008D5
:1018A0000810E000000F102020100F00001010F8AA
:1018B000000000000020203F2020000000700808E9
:1018C0000888700000302824222130000030088869
:1018D000884830000018202020110E000000C02091
:1018E00010F8000000070424243F240000F80888B2
:1018F000880808000019212020110E0000E010883F
:1019000088180000000F112020110E000038080870
:10191000C83808000000003F000000000070880880
:1019200008887000001C222121221C0000E0100801
:101930000810E0000000312222110F00000000C05A
:10194000C0000000000000303000000000000080F7
:1019500000000000000080600000000000008040E7
:101960002010080000010204081020004040404000
:101970004040400004040404040404000008102053
:101980004080000000201008040201000070480898
:101990000808F0000000003036010000C030C82800
:1019A000E810E0000718272423140B000000C038BB
:1019B000E0000000203C23020227382008F8888835
:1019C00088700000203F202020110E00C030080841
:1019D00008083800071820202010080008F8080818
:1019E0000810E000203F202020100F0008F8888811
:1019F000E8081000203F20202320180008F88888DD
:101A0000E8081000203F200003000000C030080854
:101A10000838000007182020221E020008F80800DD
:101A20000008F808203F210101213F20000808F8A4
:101A3000080800000020203F2020000000000808C7
:101A4000F8080800C08080807F00000008F888C087
:101A500028180800203F20012638200008F8080038
:101A600000000000203F20202020300008F8F8006F
:101A7000F8F80800203F003F003F200008F830C081
:101A80000008F808203F200007183F00E010080871
:101A90000810E0000F10202020100F0008F80808A0
:101AA0000808F000203F210101010000E0100808B3
:101AB0000810E0000F18242438504F0008F88888D8
:101AC00088887000203F2000030C302000708808B8
:101AD000080838000038202121221C00180808F8C6
:101AE000080818000000203F2000000008F8080047
:101AF0000008F808001F202020201F000878880018
:101B000000C83808000007380E010000F80800F887
:101B10000008F800033C0700073C03000818688031
:101B20008068180820302C03032C30200838C800A7
:101B3000C83808000000203F2000000010080808F6
:101B4000C83808002038262120201800000000FE98
:101B5000020202000000007F40404000000C30C044
:101B600000000000000000010638C0000002020270
:101B7000FE000000004040407F0000000000040222
:101B8000020204000000000000000000000000004D
:101B9000000000008080808080808080000202043D
:101BA0000000000000000000000000000000808035
:101BB000808000000019242222223F2008F80080A3
:101BC00080000000003F112020110E000000008066
:101BD00080800000000E11202020110000000080F5
:101BE0008088F800000E112020103F200000808027
:101BF00080800000001F222222221300008080F03B
:101C0000888888180020203F202000000000808065
:101C100080808000006B94949493600008F80080AA
:101C200080800000203F210000203F200080989805
:101C3000000000000020203F202000000000008065
:101C40009898000000C08080807F000008F80000A5
:101C500080808000203F24022D302000000808F8FA
:101C6000000000000020203F2020000080808080B5
:101C700080808000203F20003F20003F8080008047
:101C800080800000203F210000203F200000808055
:101C900080800000001F202020201F008080008006
:101CA0008000000080FFA12020110E0000000080B5
:101CB00080808000000E112020A0FF8080808000A6
:101CC0008080800020203F212000010000008080D3
:101CD000808080000033242424241900008080E0C8
:101CE000808000000000001F202000008080000095
:101CF00000808000001F202020103F208080800076
:101D00000080808000010E30080601008080008085
:101D1000008080800F300C030C300F0000808000AA
:101D2000808080000020312E0E31200080808000D5
:101D30000080808080818E70180601000080808085
:101D4000808080000021302C222130000000000023
:101D5000807C020200000000003F404000000000C4
:101D6000FF00000000000000FF0000000002027CF5
:101D7000800000000040403F00000000000601011C
:101D80000202040400000000000000000000000047
:101D90000000000000000000000000000000000043
:101DA0000000000000000000000000000000000033
:101DB0000000000000F0F0F0000000000000000053
:101DC00000017F010000000000000000001C1C1C3E
:101DD0000000000000008060301C8C60301C0C0093
:101DE00000000000000000000000000000000000F3
:101DF0000000000000000000000000E00000000003
:101E000000E000000086E69F86868686E69F8600C4
:101E100000011F01010101011F010100000080C03C
:101E20006020F820E0C00000000003070C18FF70DD
:101E3000E18100000000070F10107F100F07000065
:101E40008060206080000000E02000000F30203023
:101E50009F70DC371030C0000000100E0300071820
:101E6000101807000000C02020E0C00000000000A3
:101E700080E01F38E88703C43C040000070F1810F7
:101E8000100B070D1010080000808C4C380000006B
:101E90000000000000000000000000000000000042
:101EA0000000000000000000000000000000000032
:101EB000000080E0300804000000000000FEFF0188
:101EC00000000000000000000000030F1820400088
:101ED00000040830E0800000000000000000000066
:101EE00001FFFE0000000000004020180F0300006A
:101EF00000000000000000000000C0000000000022
:101F0000004266663C18FF183C666642000000000E
:101F1000000003000000000000000000000080003E
:101F200000000000001010101010FF101010101012
:101F3000000000000000030000000000000000009E
:101F40000000000000000000000000000000000091
:101F50000000000000808C4C3800000000000000F1
:101F60000000000000000000000000000010101041
:101F700010101010101010000000000000000000F1
:101F80000000000000000000000000000000000051
:101F900000000000000000000000000000001C1C09
:101FA0001C00000000000000000000000000000015
:101FB000E0380C000000000080701C0300000000EE
:101FC0000060380E0100000000000000000080C02A
:101FD00060202060C080000000FEFF0100000000C3
:101FE00001FFFE000001070E181010180E07010077
:101FF0000000808080C0E0000000000000000000C1
:1020000000FFFF000000000000001010101F1F1054
:10201000101000000080402020202060C0800000C0
:1020200000030300804020381F070000001C1A191D
:1020300018181818181F00000080C020202060C049
:1020400080000000000303001010182FE78000003C
:1020500000070F10101010180F07000000000000FC
:102060000000C0E0F000000000C0B088868180FF62
:10207000FF808000000000000010101F1F101000E3
:102080000000E060606060606060000000003F1081
:1020900008080818F0E0000000070B101010101CD2
:1020A0000F030000000080C040202020E0C000009E
:1020B00000FCFF211008080818F0E0000001070CE0
:1020C00018101010080F03000000C0E0606060608E
:1020D00060E06000000003000000E018070000005E
:1020E00000000000001F1F00000000000080C06012
:1020F0002020202060C080000087EF2C181830308E
:1021000068CF830000070F0810101010180F070089
:102110000000C0C020202020C0800000001F3F60C1
:102120004040402010FFFE0000000C1C1010100862
:102130000F0300000000000000000000000000008D
:1021400000000000000E0E0E000000000000000065
:10215000001C1C1C0000000000000000000000002B
:102160000000000000000000000C0C000000000057
:1021700000000000005838000000000000000000CF
:102180000000008040201000000010284482010060
:102190000000000000000000000001020408100020
:1021A00000000000000000000000000000848484A3
:1021B0008484848484848400000000000000000083
:1021C000000000000000102040800000000000001F
:1021D00000000000000001824428100000001008E8
:1021E000040201000000000000C0202010101010A8
:1021F00030E0C0000003030000F010080C070300EB
:10220000000000001C1C1C0000000000000000C0BA
:10221000406020202040C00000FCFF01F00E03C100
:10222000FE03807F0001070E08111110110904023E
:102230000000000080E0E000000000000000807C62
:102240004340477FF880000010181F100000000076
:10225000131F1C1020E0E02020202060C080000020
:1022600000FFFF10101010182FE78000101F1F1024
:1022700010101010180F0700000080C04020202010
:102280002060E00000FCFF010000000000000100F1
:102290000001070E181010100804030020E0E020D1
:1022A00020202040C080000000FFFF000000000050
:1022B00001FFFE00101F1F10101018080E0701006C
:1022C00020E0E020202020202060800000FFFF1080
:1022D0001010107C00000000101F1F1010101010B4
:1022E0001018060020E0E020202020206060800000
:1022F00000FFFF101010107C00000100101F1F10C5
:102300000000000000000000000080C060202020CD
:1023100040E0000000FCFF0100004040C0C1404020
:102320000001070E181010100F0F000020E0E02031
:102330000000000020E0E02000FFFF10101010104F
:1023400010FFFF00101F1F1000000000101F1F10C3
:102350000000202020E0E0202020000000000000FD
:1023600000FFFF000000000000001010101F1F10F1
:102370001010000000000000202020E0E0202020BD
:1023800000000000000000FFFF0000000060E0808F
:102390008080C07F3F00000020E0E020000020A0FF
:1023A0006020200000FFFF30187CE3C00000000028
:1023B000101F1F10000001131F1C181020E0E02048
:1023C000000000000000000000FFFF00000000000F
:1023D00000000000101F1F10101010101018060031
:1023E00020E0E0E000000000E0E0E02000FF013F2E
:1023F000FEC0E01E01FFFF00101F1000031F0300BE
:10240000101F1F1020E0E0C0000000000020E020AE
:1024100000FF0003071C78E08000FF00101F100081
:1024200000000000030F1F00000080C0602020603B
:10243000C080000000FEFF010000000000FFFE0061
:102440000001070E181010180C07010020E0E02012
:102450002020202060C0800000FFFF2020202020BE
:10246000301F0F00101F1F100000000000000000B0
:10247000000080C060202060C080000000FEFF01DE
:102480000000000000FFFE000001070E1111133CC8
:102490007C67210020E0E0202020202060C0800018
:1024A00000FFFF101030F0D0080F0700101F1F10A2
:1024B000000000030F1C10100080C06020202020AE
:1024C0004040E00000070F0C1818303060E0810039
:1024D000001F0C0810101010180F0700806020203B
:1024E00020E0E020202060800100000000FFFF00CD
:1024F0000000000100000000101F1F10000000007D
:1025000020E0E020000000000020E02000FFFF00AD
:10251000000000000000FF0000070F18101010104E
:10252000100807002060E0E02000000020E06020AC
:102530000000077FF88000807C030000000000009E
:10254000071F1C070000000020E0E02000E0E02062
:102550000020E0200007FFF8E01FFFFCE01F000064
:102560000000031F0300011F03000000002060E0C3
:10257000A0000020E0602000000000038F7CF8C66F
:10258000010000000010181E130001171F18100092
:102590002060E0E02000000020E060200000010753
:1025A0003EF8E0180700000000000010101F1F1088
:1025B0001000000000806020202020A0E0E020002B
:1025C00000000000C0F03E0F0300000000101C1FC0
:1025D00017101010101806000000000000FC040482
:1025E000040404000000000000FF000000000000E0
:1025F00000000000007F404040404000000010E02C
:10260000000000000000000000000000031C6080CB
:102610000000000000000000000000030C708000BB
:1026200000000404040404FC00000000000000009A
:10263000000000FF00000000000040404040407FDC
:102640000000000000000010080C040C081000003E
:10265000000000000000000000000000000000007A
:10266000000000000000000000000000000000006A
:10267000000000000000000000000000000000005A
:102680008080808080808080808080800000000446
:102690000408080000000000000000000000000026
:1026A000000000000000000000000000000000002A
:1026B000000000000000000000000000000098D8AA
:1026C00044642424FCF80000000F1F1810101008A8
:1026D0001F1F10180020E0F00000000000000000A4
:1026E0000000FFFF180804040CF8F00000001F0FA2
:1026F00018101010180F0300000000000000000068
:102700000000000000E0F8180404043C3800000059
:1027100000030F0C1010101008060000000000004D
:1027200000000020E0F0000000E0F81C04040408B1
:10273000FFFF000000030F18101010081F0F080003
:102740000000000000000000000000000000E0F8B1
:10275000484444444C7870000000030F0C181010DB
:10276000100804000000000080C0602020E0C000CD
:1027700000040404FFFF040404040000000010101F
:102780001F1F1010100000000000000000000000DB
:1027900000000000000070F88C04048CF874040C35
:1027A000007076CF8D8D8D89C87870000020E0F0A4
:1027B00000000000000000000000FFFF0804040407
:1027C000FCF8000000101F1F100000101F1F100059
:1027D0000000000000606000000000000000040431
:1027E00004FCFC000000000000001010101F1F106F
:1027F00010100000000000000000006060000000F9
:1028000000000000040404FCFC0000000000C0C044
:102810008080C07F3F0000000020E0F0000000004A
:10282000000000000000FFFF80C0F41C0404000052
:1028300000101F1F1100031F1C101000000020209B
:1028400020E0F000000000000000000000FFFF009A
:102850000000000000001010101F1F1010100000DA
:1028600000000000000000000000000004FCFC0864
:1028700004FCFC0804FCFC00101F1F10001F1F10AC
:10288000001F1F10000000000000000000000000FA
:102890000004FCFC08080404FCF8000000101F1FE2
:1028A000100000101F1F10000000000000000000BA
:1028B0000000000000E0F0180C04040C18F0E00028
:1028C00000030F0C101010100C0F0300000000008C
:1028D00000000000000000000004FCFC08040404E8
:1028E0000CF8F0000080FFFF889010101C0F030010
:1028F00000000000000000000000000000E0F81CE4
:1029000004040408F8FC000000030F18101090885D
:10291000FFFF800000000000000000000000000039
:10292000040404FCFC100804040C0C001010101F1C
:102930001F10101000000000000000000000000048
:102940000000000000003078CCC48484840C1C009B
:1029500000001E1810101011190F060000000000D2
:1029600000C000000000000000040404FFFF040495
:1029700004000000000000000F1F1010100C0000E9
:102980000000000000000000000000000004FCFE49
:1029900000000004FCFE000000000F1F18101008CB
:1029A0001F0F0800000000000000000000000000F1
:1029B00000040C3CFCC40000C43C0C0400000000FB
:1029C000010F1E0E010000000000000000000000CA
:1029D00000000000043CFCC400E47CFC84807C0417
:1029E0000000071F070000071F070000000000008D
:1029F00000000000000000000004041C7CE4C0345F
:102A00001C0404000010101C1601131F1C181000D9
:102A100000000000000000000000000000040C3C6A
:102A2000FCC400C43C0404000000C080C1370E0197
:102A30000000000000000000000000000000000096
:102A400000001C0404C4F47C1C0400000000101CE2
:102A50001F17111010180E0000000000000000F8F1
:102A60000C04000000000000001028EF000000002F
:102A7000000000000000003F604000000000000077
:102A80000000FF0000000000000000000000FF0048
:102A900000000000000000000000FF000000000037
:102AA0000000040CF800000000000000000000001E
:102AB000EF28100000000000000040603F00000010
:102AC0000000000000180602020408102020300850
:102AD00000000000000000000000000000000000F6
:102AE00000000000000000000000000001020304DC
:102AF00000000000000000000000000000000000D6
:102B000000000000000000000000000000000000C5
:102B100000000000000000000000000000000000B5
:102B200000000000000000000000000000000000A5
:103090000000000000000000808080808080000030
:1030A000000000C0E0E0E0E0C0C000000000000060
:1030B0000000000000000000000000000000000010
:1030C0000000000000000000000000000000000000
:1030D000000000000000000000007EFEFEFEFEFE7C
:1030E000FE00000080FEFEFEFEFEFEFEFC00000074
:1030F00000FCFEFEFEFEFE3E0000000000000000A0
:1031000080808080808000000000000000000000BF
:10311000000080F8FEFEFEFEFEFEFEFEF0800000D7
:10312000000000000000000000000080808080801F
:1031300080000000000000F8F8F8F8F8F8F8000047
:103140000000000000000000000000000000E0F0AF
:10315000F8FCFCFEFE7E7E3E3E7E7EFEFCFC783071
:1031600000000000F8F8F8F8F8F8F8000000000097
:10317000000000000000000000000000000000004F
:10318000000000000000000000000000808080803F
:103190008000FFFFFFFFFFFFFF000000030F1F1F66
:1031A0001F1F0F0F00000000000000000080808043
:1031B000808080800000000000000000000000000F
:1031C00000000000000000000000000000000000FF
:1031D00000000000003FFFFFFFFFFFFC00C0FFFFFB
:1031E000FFFF7FFFFFFFFFFF8000FEFFFFFFFFFFEE
:1031F0000F000000F0F8FEFEFFFF7F1F0F0F1FFF04
:10320000FFFFFEFCF8C000000000C0FCFFFFFFFF56
:103210007F071FFFFFFFFFFFF88000000000C0F0E6
:10322000FCFEFFFFFF7F1F1F1F1F3F3F3F0E041FBE
:103230001FFFFFFFFFFFFFFF1F1F1F1F00000000FA
:1032400000000000000000001F7FFFFFFFFFFFFCE9
:10325000F8F8F0F0E0E0C1C08000001F1F1FFFFF82
:10326000FFFFFFFFFF1F1F1F0F000000FFFFFFFFFB
:10327000FFFF00000000FFFFFFFFFFFFFF00000057
:10328000C0F8FCFEFFFFFF7F1F1F1F3FFFFFFFFF78
:10329000FFFFFF00000000FFFFFFFFFFFFFF000038
:1032A00000C0F8FCFEFFFFFF3F1F1F1F3FFFFFFF97
:1032B000FEFCF8E00000000000000000000000003C
:1032C00000000000000000000000000000000000FE
:1032D0000FFFFFFFFFFFFCFFFFFFFF1F0001FFFFCE
:1032E000FFFFFFFEFFFFFFFFFF070000001EFFFFC5
:1032F000FFFFFFFFDF1F1F1F1F1F1F9F9F1F1F1F9E
:103300000000E0FEFFFFFFFFFFFFFCFCFCFDFFFFF6
:10331000FFFFFFFFFCC00000FFFFFFFFFFFFFF807C
:103320000000000000800000000000FFFFFFFFFF22
:10333000FFFF00000000000000000000000000008F
:10334000000080C0C0800101030303070FFFFFFFDF
:10335000FFFFFFFF70000000FFFFFFFFFFFFFF0008
:10336000000000000000FFFFFFFFFFFF00000080E3
:10337000FFFFFFFFFFFFFF000000FFFFFFFFFFFF5A
:10338000FF8000000000FFFFFFFFFFFFFF000000C5
:1033900000FFFFFFFFFFFFFF000000FFFFFFFFFF39
:1033A000FFFF8000000000FFFFFFFFFFFFFF0000A6
:1033B000000000000000000000000000000000000D
:1033C0000000000000000000000000073F3F3F3FFA
:1033D0003F3F3F3F0F000000003F3F3F3F3F3F3F29
:1033E0003F3F01000000000001070F1F1F3F3F3F4C
:1033F0003E3E3E3E3F3F1F1F0E00303E3F3F3F3FA1
:103400003F1F01000000000000033F3F3F3F3F3FE0
:103410003C000003070F1F3F3F3F3F3E3E3F3F3F03
:103420001F1E080000030F1F3F3F3F3F3F3E3F3F2F
:103430001C18000000000000000000070F1F1F3FC5
:103440003F3F3F3E3E3F3F3F3F1F1F0F07030000F0
:103450000000070F1F3F3F3F3F3E3F3F3F1C000024
:103460000F1F3F3F3F3F3F3E3F1F1F3F3F3F3F3FFD
:103470003F00000000070F1F3F3F3F3F3F3E3F1F01
:103480001F3F3F3F3F3F3F000000003F3F3F3F3F68
:103490003F3F0000000003070F1F3F3F3F3F3E3EFE
:1034A0003F3F3F1F1F0F030000000000000000000F
:1034B000000000000000000000000000000000000C
:1034C00000000000000000000000000000000000FC
:1034D00000000000000000000000000000000000EC
:1034E00000000000000000000000000000000000DC
:103BC000C0C0C0C0C0000080C0C0C0C08000000035
:103BD00000000000000000000000000000000000E5
:103BE00000000000000000000000000000000000D5
:103BF00000000000000000000000000000000000C5
:103C000000000000000000000000000000000000B4
:103C100000000000000000000000000000000000A4
:103C20000000000000000000000000000000000094
:103C30000000000000000000000000000000000084
:103C40000000000000000000000000000000000074
:103C5000000000C0C0C0C0C0C000000000000000E4
:103C6000000000000000000000C0C0C0C0C0000094
:103C70000000000000000000000000000000000044
:103C8000000000000000000000000000000C1E1FEB
:103C90001F0F0F9FFFFFFEFEF80000000000000056
:103CA00038787C7E3EFFFFFFFFFF00040E1E1F8F53
:103CB0008F8FFFFFFFFEFC000000737F3F1F0F0090
:103CC00000317B7F3F1F070000000000000000FF65
:103CD000FFFFFFFF8787878787070000F0F0F0F07E
:103CE000F0F070F8F8F0F0E0800030F0F0F0787864
:103CF000F8F0F0F0E0800000F0F0F0F0F0F070F894
:103D0000F8F0F0E0800080E0F0F0F0F878F0F0F00B
:103D1000E0C00000F0F0F0F0F0F0F0F0F010000083
:103D20000000000000FFFFFFFFFFFFFEC0E0FFFFFD
:103D3000FFFFFFFFFF000080C0E0F0F0F078F8F038
:103D4000F0F0E0C00000C0E0F0F0F8F870FFFFFF16
:103D5000FFFFFF0000F0F0F0F0F000F0F0F0F0F006
:103D6000F00000FFFFFFFFFF000080C0E0F0F0F870
:103D700078F8F0F0F0E080000000000000000000A3
:103D80000000000000000080C0F0F8FCFEFFBF9FB4
:103D900087838000C0C0C0C0C0800000000000FF5A
:103DA000FFFFFFFF0080C0C0C0C78787CFFFFFFFB6
:103DB000FEF800000000000000000000000000000D
:103DC000000000000000000000FFFFFFFFFF8787EA
:103DD000878787800000FFFFFFFFFF8080E1FFFFF4
:103DE000FFFF7F40F8FCFCFEFE9ECFFFFFFFFFFFC2
:103DF0000000FFFFFFFFFF8080E1FFFFFFFF7F006C
:103E0000FFFFFFFFFFDC9C9D9FDFDF9F1F00FFFF89
:103E1000FFFFFF0301000000000000000000FFFFA3
:103E2000FFFFFF0FFFFFFFFFFFFF0FFFFFFFFFFC85
:103E3000007FFFFFFFFFE18080FFFFFFFFFF1C0807
:103E4000FFFFFFFFFF8080FFFFFFFFFFFF0000FF7E
:103E5000FFFFFFFF80FFFFFFFFFFFF0000FFFFFFEF
:103E6000FFFF80007FFFFFFFFFDC9C9C9FDFDF9F49
:103E70001F00000000000000000000000000000023
:103E800000070707070707070707070707000307D4
:103E900007070703000000000007070707070001E6
:103EA00003030707070707070703010000000000D7
:103EB0000000000000000000000000000000000002
:103EC00000000007070707070707070707070000A5
:103ED000FFFFFFFFFF0707070707030100000307B6
:103EE000070707070703070707070000FFFFFFFF94
:103EF000FF07070707070301000000010307070783
:103F0000070707070303000007070707070000006C
:103F1000000000000000000007070707070001017C
:103F20000101010000070707070700000103070759
:103F30000707070707030300000001030707070738
:103F40000707070707070700000307070707070713
:103F50000707070707000003070707070707000110
:103F60000307070707070707030300000000000017
:103F70000000000000000000000000000000000041
:103F80000000000000000000000000000000000031
:103F90000000000000000000000000000000000021
:103FA0000000000000000000000000000000000011
:104580000000000070F0F8FC7CFEFEFEFEFE00184D
:104590003C3C3E3E1E1EFEFEFEFCF800183C3E3E2D
:1045A0001E1E3EFEFEFCFCF000000000000000E0CD
:1045B000E0E0E0E0C080E0E0E0E0E00000000000DB
:1045C00000183C3C3E3E1E1EFEFEFEFCF80000FEB7
:1045D000FEFEFEFE9E9E9E9E1E1E0000E0F8FCFE5D
:1045E000FE7E1E3EFEFEFCF8E00000000000000023
:1045F00000FEFEFEFEFEFE0E0E0E0E0E0E00000073
:10460000000000000000000000FEFEFEFEFE0000B4
:104610000000000000FEFEFEFEFE000000FEFEFEAA
:10462000FEFEFEFCE000FEFEFEFEFE0000FEFEFEC4
:10463000FEFEC0E0F8FCFEFE3E1E0600000000008C
:10464000000000000000000000000000000000006A
:10465000000000000000000000000000000000005A
:10466000000000000000000000000000000000004A
:10467000000000000000000000000000000000003A
:10468000000000FFFFFFFFFF000080C0E0F0FCFE25
:104690007F3F1F0F03000080E0F0F8FCFF7F3F0F1B
:1046A00007010000000000000000C1E7FFFFFFFF5E
:1046B000FFFFF7C1000000000000000080C0E0F034
:1046C000FCFE7F3F1F0F0300008787878707078F48
:1046D000FFFFFFFFFC007FFFFFFFFFC00080FFFF29
:1046E000FFFFFF0000000000000000FFFFFFFFFFD2
:1046F000FF0F0F0F0F0F00001E1E1E1E1E1E1E1E80
:104700001E0000FFFFFFFFFF00000000000000FF91
:10471000FFFFFFFF000000FFFFFFFFFF3FFFFFFF66
:10472000FFFFFFFFFF0000FFFFFFFFFF1F7FFFFFF7
:10473000FFF8E0C0000000000000000000000000E2
:104740000000000000000000000000000000000069
:104750000000000000000000000000000000000059
:104760000000000000000000000000000000000049
:10477000000000000000000000000000000F0F0F0C
:104780000F0F00000F0F0F0F0F0F0F0F0F0F0F075F
:104790000F0F0F0F0F0F0F0F0F0F0F0F0000000065
:1047A00000000C0F0F0F0F0F0101070F0F0F0F0C61
:1047B0000000000000000F0F0F0F0F0F0F0F0F0F63
:1047C0000F070307070F0F0F0F0F0F0F070301004E
:1047D0000003070F0F0F0F0F0F0F0703000000005C
:1047E00000000000000F0F0F0F0F0F0F0F0F0F0F24
:1047F0000F0000000000000000000000000F0F0F7D
:104800000F0F0F0F0F0F0F0F000F0F0F0F0F0000E5
:10481000000F0F0F0F0F00010F0F0F0F0F0F0F00E3
:10482000000F0F0F0F0F000001030F0F0F0F0F0CE2
:104830000000000000000000000000000000000078
:104840000000000000000000000000000000000068
:104850000000000000000000000000000000000058
:104860000000000000000000000000000000000048
:104870000000000000000000000000000000000038
:104880000000000000000000000000000000000028
:104890000000000000000000000000000000000018
:1048A0000000000000000000000000000000000008
:1048B00000000000000000000000000000000000F8
:1048C00000000000000000000000000000000000E8
:1048D00000000000000000000000000000000000D8
:1048E00000000000000000000000000000000000C8
:1048F00000000000000000000000000000000000B8
:1049000000000000000000000000000000000000A7
:104910000000000000000000000000000000000097
:104920000000000000000000000000000000000087
:104930000000000000000000000000000000000077
:104940000000000000000000000000000000000067
:104950000000000000000000000000000000000057
:104960000000000000000000000000000000000047
:104970000000000000000000000000000000000037
:104980000000000000000000000000000000000027
:104990000000000000000000000000000000000017
:1049A0000000000000000000000000000000000007
:1049B00000000000000000000000000000000000F7
:1049C00000000000000000000000000000000000E7
:1049D00000000000000000000000000000000000D7
:1049E00000000000000000000000000000000000C7
:1049F00000000000000000000000000000000000B7
:104A000000000000000000000000000000000000A6
:104A10000000000000000000000000000000000096
:104A20000000000000000000000000000000000086
:104A30000D0A57654163742053747564696F204390
:104A40006F726520426F6172640D007765616374F7
:104A500073747564696F2E74616F62616F2E636F1A
:104A60006D0D00776561637473747564696F2E6191
:104A70006C69657870726573732E636F6D0D0000DD
:104A8000A04A00080000002008000000680F00088D
:104A9000A84A00080800002058230000780F0008EA
:084AA0000000000000D8B80579
:04000005080000FDF2
:00000001FF
